:020000040000FA
:02000000092ACB
:08000800A000030E8312A10009
:100010002608820020342034203420342034203438
:100020006534733463342E34613473346D34203466
:10003000563431342E3435342034203420342034B6
:100040004534533443344234203420342034203473
:10005000B801B901BA01B90AB601B7010310B50D6B
:10006000B80D03183628B90DBA0D2E28B80CB50CEA
:100070003508B3023808031C013EB402031C4C28A7
:100080003908B6043A08B7040310BA0CB90C0318BF
:100090000800B80CB50C38283508B3070318B40AA3
:1000A0003808B4074428B601B7013508B800381C31
:1000B0005F283308B60734080318013EB70703105A
:1000C000B80C3808031908000310B30DB40D5728F5
:0C00D000313E8200713E8200B13E820091
:1002000085010000062A27088500082200008501D4
:10021000062A2708850005292708850000000B29E4
:10022000270885000E2927088500000012292708C5
:100230008500152927088500000019292708850051
:1002400000001C2927088500042A000085010822D7
:10025000292927088500042A000085010822302961
:100260002729003400340034033409340C341034AA
:10027000133417341A341E34F134F134F134F134B8
:10028000F134F134F134F134F134F134F134F13446
:10029000F134F134F134F134F134F134F134F13436
:1002A000F134F134F134F134F134F134F134F13426
:1002B000F134F134F134F134F134F134F134F13416
:1002C000F134F134F134F134F134F134F134F13406
:1002D000F134F134F134F134F134F1342C34253487
:1002E000223400340034003400340034003400344C
:1002F0000034003400340034FB34FA34F834F7347A
:10030000F534F334F134EF34ED34EB34E934E734DD
:10031000E434E234DF34DC34D934D634D234CF346C
:10032000CB34C734C334BE34B934B434AE34A83457
:10033000A1349A34923489347F34753469345C340E
:100340004D343C3429341334093409340934093424
:1003500009340934093409340934093408340834B7
:100360000834083408340834C834C834C834C834AD
:10037000C834C834C834C834C934C934C934C93499
:10038000C934C934C934C934C934C934C934C93485
:10039000C934C934C934C934C934C934C934C93475
:1003A000C934C934C934C934C934C934C934C93465
:1003B000C934C934C934C934C934C934C934C93455
:1003C000C934C934C934C934CD34D334D934DE3412
:1003D000E434E934EE34F334F834FC3400340034DB
:1003E0000034A218F829A214000085012908FD296B
:1003F000270885002808A210000081000B11210E9B
:100400008300A00E200E09002808FD292908FD29D7
:1004100008008316FF239000831201308A008501B3
:100420008316A83099008312033099008316303068
:1004300002389F001030950000308100DF30FB391A
:10044000FE3985008312FF3081008B16A201143023
:10045000A300A501A701A801A901F130A600FF3062
:10046000AF00B000B100B2008B17F5222218352A78
:100470004308BC00BE004208BB00403EBD0003185C
:10048000BE0AF5222218412A42083D024308031CF5
:10049000013E3E020318412A4208BD004308BE0047
:1004A0003B083D02B300AD003C08031C013E3E0288
:1004B000B400AE004030B50028203608AC00B300D0
:1004C000B40153203608AD023708031C013EAE02CA
:1004D0000310AE0CAD0C3B08AD073C080318013E01
:1004E000AE07F5222218712A3D0842023E08031C7D
:1004F000013E430203184C2A4208B3004308B400EB
:1005000020230038031D712A8B17DB22E822DB220F
:100510008B17A501A701CB222308A40019232218B9
:100520008C2A6820003C031D8C2AA40B8E2A0130E3
:10053000A300A7018501A501CB222030A700192324
:100540002218892A25020319B12A0318AB2AA50A01
:10055000CB2222119F2A221DAF2AA502CB222215CF
:100560009F2A22112608003C031D9F2A851D9F2AD1
:100570000130A7000130A500CB2219232218892AB7
:100580006820003C031D992A250A3F3C031CBD2A14
:10059000A50ACB22BD2A25086A20AA0025086C20BE
:1005A000AB00250868208B12A6002A08A8002B089B
:1005B000A9008B160800C830BF0020308500082233
:1005C0000822082208228501EE22BF0BDD2A08003E
:1005D000C830BF00EE22BF0BEA2A080064003230A8
:1005E000C0000822C00BF12A08003423221808009A
:1005F0000530C1000E08C2000F08C30034232218C2
:1006000008004208FD3EB3004308031CFF3EB4004F
:1006100033080E02B3003408031C013E0F02B4007D
:10062000031DF52A073033020318F52AC10BFE2AF1
:1006300008003423221800340E08B3000F08B40059
:100640002D08B3022E08031C013EB402031C003423
:100650002C08B5002820B708031D3F34403036026F
:1006600003183F343608080022104030C4001B3005
:10067000C5008E018F0141309000592322180034AB
:100680000E080F0403193D2B59232218003409309A
:100690000F020318532B051E442B900103300F0249
:1006A000031C392B0800592322180034051E532B34
:1006B000392B6400C40B0800C50B08002214080085
:1006C0003108B2003008B1002F08B0001E08AF009A
:1006D000C600C7013008C6070318C70A3108C60795
:1006E0000318C70A3208C6070318C70AC70CC60C86
:0806F000C70CC60C4608080007
:02400E00CC3FA5
:00000001FF
